:10000300EFD394077480948040037F012212027A15
:10001300FED394037480948040037F0222EF7044E4
:10002300EE700B900001120293F452935294120259
:100033007A6401700B9000011202934293F452947C
:1000430012027AFE6402700A900001120293429334
:100053004294EE6403700D900001120293FEF45279
:1000630093EE4294EF6401704612027AFE700B9095
:100073000001120293F452915292EE6401700B90BC
:1000830000011202934291F4529212027A640270B6
:100093000A9000011202934291429212027A64037F
:1000A300700D900001120293FEF45291EE4292EF12
:1000B3006402704612027AFE700B900001120293E2
:1000C300F452955296EE6401700B90000112029364
:1000D3004295F4529612027A6402700A9000011259
:1000E30002934295429612027A6403700D900001C6
:1000F300120293FEF45295EE4296EF640370461299
:10010300027AFE700B900001120293F452B152B2C4
:10011300EE6401700B90000112029342B1F452B2EB
:1001230012027A6402700A90000112029342B142F1
:10013300B212027A6403700D900001120293FEF46E
:1001430052B1EE42B2EF6404704612027AFE700BB3
:10015300900001120293F452B352B4EE6401700B97
:1001630090000112029342B3F452B412027A640271
:10017300700A90000112029342B342B412027A64ED
:1001830003700D900001120293FEF452B3EE42B4D9
:10019300EF6405704612027AFE700B9000011202A2
:1001A30093F452C952CAEE6401700B90000112021B
:1001B3009342C9F452CA12027A6402700A9000018F
:1001C30012029342C942CA12027A6403700D90006C
:1001D30001120293FEF452C9EE42CAEF640670465E
:1001E30012027AFE700B900001120293F452CB526A
:1001F300CCEE6401700B90000112029342CBF452D7
:10020300CC12027A6402700A90000112029342CB6C
:1002130042CC12027A6403700D900001120293FE25
:10022300F452CBEE42CCEF6407704912027AFF7EA0
:1002330000700B900001120293F452E152E2EF645A
:10024300014E700B90000112029342E1F452E2124C
:10025300027A6402700A90000112029342E142E2C0
:1002630012027A6403700D900001120293FFF4529C
:07027300E1EF42E27F0022EF
:1002EE00750903E4F508FB7A0079087F050200031F
:1002C0001202EEB2C87FFA7E001202D7B2C97FFADC
:0702D0007E001202D780EC52
:1002D7007D607C09ED1D70011C144C70F7EF1F70D9
:0602E700011E144E70EA36
:0102ED0022EE
:030000000202FEFB
:0C02FE00787FE4F6D8FD7581090202C08B
:10027A00BB010689828A83E0225002E722BBFE0282
:09028A00E32289828A83E49322B5
:10029300BB010CE58229F582E5833AF583E0225020
:1002A30006E92582F8E622BBFE06E92582F8E2226A
:0D02B300E58229F582E5833AF583E4932284
:00000001FF
